:020000000C28CA
:08000800B6000308B700370839
:100010008300B60E360E09008B0183168117FF3060
:10002000850086018312ED22303086008615ED2290
:100030008611303086008615F02286113030860019
:100040008615F0228611203086008615F32286114F
:100050002830AB00A4220830AB00A4220130AB0052
:10006000A4220630AB00A4220C30AB00A4228519D8
:100070003A2858218901E5220808A300E52208084A
:10008000A400E5220808A500E5220808A6002830FB
:100090008C0001308D00D6308E0000308F0007229A
:1000A0003722B721ED21ED210508B30003303305D8
:1000B000B200B0014030AF00B401B9012E21B31D30
:1000C0007C289D019C019B0101309A003319722804
:1000D000E8309A0003309B00722803109A0D9B0DA4
:1000E0009C0D9D0DAF0DB00D031C6D28B4187A2822
:1000F00007218F28CB208F28B41888280430B90214
:10010000DF303907031C86282030B900B9208F283A
:100110000430B907DF3039070318B901B9200722C5
:100120003722B721ED215E28820700341B34773453
:100130004034003435346734E03400346A34CF342A
:10014000C03400349A341D3420340034D5349F3404
:10015000803401341334B2342034013440346F34E9
:10016000403401347B34CA3490340134AB343F34EE
:100170000034390894208F00B90A390894208E0081
:10018000B90A390894208D00B90A390894208C00E6
:100190000330B90208001A088C07031CD4288D0FFD
:1001A000D4288E0FD4288F0A1B088D07031CDB2848
:1001B0008E0FDB288F0A1C088E07031CE0288F0A8D
:1001C0001D088F07FE300F070318FE2801300F02AD
:1001D000031C062936300E070318FE28C9300E020C
:1001E000031C06293C300D070318FE28C3300D02FE
:1001F000031C062980300C02031C062980308C0069
:10020000C3308D00C9308E0001308F0008009A097C
:100210009B099C099D099A0F12299B0F12299C0F7B
:1002200012299D0ACB208F1B27298F08031D2D29FA
:100230008E08031D2D2903300D02031C2729FC30D5
:100240000D0703182D2917300C0703182D29E83046
:100250008C0003308D008E018F010800B00140300A
:10026000AF006400B01B38290830AF070318B00A8C
:100270000508B30003303305B100320603193129F4
:100280000310B20D3108B20632080239B500340647
:1002900003194F293508B4003108B2003129B218CA
:1002A0005329B40155290230B4003108B2000800C6
:1002B00080308C0096308D0098308E0000308F009A
:1002C0000630A300F030A400CA30A5002330A600F9
:1002D00007223722C430AB00A4224330AB00BE2239
:1002E0004130AB00BE224C30AB00BE22B721ED2125
:1002F0002E219D019C019B0110309A003319822907
:1003000080309A000000B41890299A099B099C0932
:100310009D099A0F90299B0F90299C0F90299D0A67
:100320001A08A307031C9929A40F9929A50F992935
:10033000A60A1B08A407031CA029A50FA029A60A2A
:100340001C08A507031CA529A60A1D08A607B31D9E
:100350007629890123088800D82224088800D82219
:1003600025088800D82226088800D8220800950190
:1003700096019701980199012030A0002308A70059
:100380002408A8002508A9002608AA000310271C95
:10039000E0290C089607031CD229970FD229980F41
:1003A000D229990A0D089707031CD929980FD92932
:1003B000990A0E089807031CDE29990A0F08990765
:1003C000990C980C970C960C950CAA0CA90CA80CDF
:1003D000A70CA00BC629990108001530840000085D
:1003E000A2000830A100A20C031CFA298617861669
:1003F0008612FD29861386168612A10BF329840A1C
:100400001A300402031CEF290614061008002030DD
:100410009E009001910192019301940103108C0DB3
:100420008D0D8E0D8F0D03180C14900D910D920DE6
:10043000930D940D9E03031D1E2A080010308400A6
:100440002A22840A2A22840A2A22840A2A22840A44
:100450002A220E2A00089F0033309F0703019F1DA8
:1004600003389F1F30389F021F088000080081302A
:10047000AB00A4221308AB00F030AB05AB0E30305C
:10048000AB04BE221308AB000F30AB053030AB0419
:10049000BE222C30AB00BE221208AB00F030AB0500
:1004A000AB0E3030AB04BE221208AB000F30AB05F0
:1004B0003030AB04BE221108AB00F030AB05AB0E00
:1004C0003030AB04BE222E30AB00BE22C030AB00B9
:1004D000A4221108AB000F30AB053030AB04BE22B4
:1004E0001008AB00F030AB05AB0E3030AB04BE22D1
:1004F0001008AB000F30AB053030AB04BE2220300B
:10050000AB00BE226B30AB00BE224830AB00BE2237
:100510007A30AB00BE22080086018316F0308600D8
:10052000831286100615FF30AD0086150608AC0054
:10053000861100000000861500008611AD03031926
:10054000A32AAC1B952A08008C2286018316003052
:1005500086008312861006110F3086052B08F039AD
:1005600086048615000086110F308605AB0E2B0819
:10057000F039860486150000861108008C22860159
:100580008316003086008312861406110F3086050C
:100590002B08F03986048615000086110F30860579
:1005A000AB0E2B08F0398604861500008611080072
:1005B0008316081555308900AA30890088148818D8
:1005C000DF2A08118312890A08008316081483128F
:1005D000890A0800FF30AD00F82A8030AD00F82A03
:1005E0004030AD00F82A2030AD00F82A1030AD00C0
:0E05F000FF30AE00AE0BFA2AAD0BF82A080061
:084000007F007F007F007F00BC
:02400E00FD3F74
:1042000070009100CA0023000000000000000000C0
:10421000000000000000000000000000000000009E
:10422000000000000000000000000000000000008E
:10423000000000000000000000000000000000007E
:10424000000000000000000000000000000000006E
:10425000000000000000000000000000000000005E
:10426000000000000000000000000000000000004E
:10427000000000000000000000000000000000003E
:00000001FF
